:020000040800F2
:100000000005002011020008151100081911000850
:100010006D110008191100084111000813020008B1
:10002000130200081302000813020008F933000845
:10003000130200081302000813020008130200084C
:10004000130200081302000813020008130200083C
:100050001302000813020008E538000811390008EF
:100060003D39000869390008953900081302000875
:10007000130200081302000813020008130200080C
:10008000130200081302000813020008A12200084E
:100090001123000871230008D1230008C13900088A
:1000A00013020008130200081302000813020008DC
:1000B000F5360008130200081302000813020008B6
:1000C00013020008130200081302000813020008BC
:1000D00013020008A9270008BD2700081302000822
:1000E000293A00081302000813020008130200084E
:1000F000130200081302000813020008130200088C
:10010000130200081302000813020008130200087B
:10011000130200081302000813020008130200086B
:10012000130200081302000813020008130200085B
:10013000130200081302000813020008130200084B
:10014000130200081302000813020008130200083B
:10015000130200081302000813020008130200082B
:10016000130200081302000813020008130200081B
:10017000130200081302000813020008130200080B
:1001800013020008130200081302000813020008FB
:1001900013020008130200081302000813020008EB
:1001A00013020008130200081302000813020008DB
:1001B00013020008130200081302000813020008CB
:1001C00013020008130200081302000813020008BB
:1001D00013020008130200081302000813020008AB
:1001E000D0400B1CD1409C46203AD3401843524289
:1001F00063469340184370479140031C90409C46CF
:10020000203A9340194352426346D3401943704702
:1002100002E000F000F8FEE772B6394880F3088883
:10022000384880F3098838484EF60851CEF200016C
:10023000086040F20000CCF200004EF63471CEF2BD
:1002400000010860BFF34F8FBFF36F8F40F20000D3
:10025000C0F2F0004EF68851CEF200010860BFF304
:100260004F8FBFF36F8F4FF00000E1EE100A4EF694
:100270003C71CEF200010860062080F31488BFF3C1
:100280006F8F03F0F7F803F0D5F94FF055301F49A1
:100290001B4A91423CBF41F8040BFAE71C49194A3A
:1002A00091423CBF41F8040BFAE71A491A4A1B4B2A
:1002B0009A423EBF51F8040B42F8040BF8E70020C5
:1002C0001749184A91423CBF41F8040BFAE703F082
:1002D000D5F803F003FA144C144DAC4203DA54F889
:1002E000041B8847F9E700F03FF8114C114DAC4270
:1002F00003DA54F8041B8847F9E703F0BDB800009F
:10030000000500200025002000000008000100205A
:1003100000050020A0460008002500207C250020C4
:1003200080250020DC420020E0010008E0010008F8
:10033000E0010008E00100082DE9F04F2DED108AE2
:10034000C1F80CD0C3689D46BDEC108ABDE8F08FA3
:10035000002383F311882846A047002002F0AAFD5D
:1003600002F050FD00DFFEE7304B6FF0160270B573
:100370001A70032200245A7007229C70DC701C71D2
:100380005C719C71DC711C725C729A72DC7203F09D
:1003900009F8064603F02AF8054678B9244B9E4230
:1003A0002ED001339E422DD0224B26F0FF029A42DE
:1003B0002BD1F0B200F03AFA42F2107400F066FC71
:1003C00000F03AFA064618B324BB2E46002002F08D
:1003D000F3FF194B1B691B071FD40EB100F02EF859
:1003E00000F076FC00F01CFE00F0D4FE0546B4B12F
:1003F00000F0D0FE401BA04211D900F01FF8F3E737
:100400000446DBE704460125D8E74FF47A74D5E7C4
:100410000446DBE74FF47A74D8E70024E0E700F005
:10042000ADFC4FF47A7002F04BFDE0E78025002030
:10043000010007B0000008B00004024010B51C4BDA
:100440001C4953F8042F013200D110BD8B42F8D162
:10045000194C1A4B22689A4228D9194B9B6803F110
:10046000006303F580339A4220D2002000F0F2FDB1
:10047000144B0220187000F021FE134B1A6C00225E
:100480001A64196E1A66196E596C5A64596E5A6656
:100490005B6E72B60D4A0E4B13601B6822682021FA
:1004A00081F311889D4683F30888104710BD00BF73
:1004B000FCFF00081C00010804000108FFFF000801
:1004C000802500208C2500200038024008ED00E047
:1004D0000000010809490B6849F269009AB21B0C37
:1004E00000FB0233064A0B60136844F2506198B275
:1004F0001B0C01FB0030106080B2704714250020F7
:100500001025002010B500211022044600F0F2FD55
:10051000034B03CB206061601868A06010BD00BF72
:10052000107AFF1FF0B51F4CBBB000F033FEA3687C
:10053000C31AF92B30D906AD2346A060282200212A
:10054000284601F0B3FB04F10E0000F0CBFD0023C0
:10055000C6B2591D5F1CDBB2B3424FEAC10107DAD4
:100560000E3323440822284601F0A0FB3B46F0E767
:10057000012303930823207B02930B4B0193C1F3C8
:10058000CF013023059100930146049503A3D3E9DD
:100590000023064801F05AF93BB0F0BD78F6339FCE
:1005A00093CACD8DC8350020D5350020A435002054
:1005B00070B50D4614461E4601F0EEF850B9022EF5
:1005C0000ED1012C0CD112A3D3E90023C5E90023DD
:1005D000012070BD052C14D003D8012C09D00020B7
:1005E00070BD282C09D0302CF9D10BA3D3E90023FE
:1005F000ECE70BA3D3E90023E8E70BA3D3E900233F
:10060000E4E70BA3D3E90023E0E700BFAFF30080EA
:10061000401DA12026812A0B78F6339F93CACD8DE9
:100620009E6AC421818A46EE26417272DF25D7B7C1
:10063000F017304A39059E5638B504460D46034634
:1006400020222846002101F031FB22792346032A8B
:1006500028BF032203F8042F28460222202101F09C
:1006600025FB62792346072A28BF072203F8052FB6
:1006700028460322222101F019FBA2792346072AEA
:1006800028BF072203F8062F28460322252101F060
:100690000DFB284604F108031022282101F006FB77
:1006A000382038BD2DE9F04FFFB01FAD0CAE40F241
:1006B000791280460F462846002100F01BFD482293
:1006C0000021304600F016FD00F064FD554B4FF45C
:1006D0007A72B0FBF2F0186093E80700012386E815
:1006E000070033740DF1520000237374FFF70AFF03
:1006F00006AB18464C4903F04DFA162230642946E1
:10070000304686F83C20FFF797FF10AB04460146C1
:100710000822284601F0CAFA0822A1180DF1410367
:10072000284601F0C3FA0DF14203082204F110013A
:10073000284601F0BBFA11AB202204F1180128462B
:1007400001F0B4FA12AB402204F13801284601F05E
:10075000ADFA14AB082204F17801284601F0A6FA9C
:100760000DF15103082204F18001284601F09EFAA0
:1007700004F1880A0DF1520904F5847B4B46514679
:10078000082228460AF1080A01F090FAD34509F137
:100790000109F3D119AB08225946284601F086FA1F
:1007A00004F588744FF0000996F834304B4510D8A2
:1007B0004FF0000996F83C304B4515D9336C214673
:1007C0004B440822284601F071FA083409F1010966
:1007D000F0E7B36B21464B440822284601F066FA45
:1007E000083409F10109DFE7E31DC3F3CF03F97E04
:1007F0000593002304950393BB7E029319370123CD
:100800000093019705A3D3E90023404601F01EF8A9
:100810007FB0BDE8F08F00BFAFF300809E6AC421B7
:10082000818A46EE90250020303D0008014B18706B
:10083000704700BF0425002070B5274B1B7B88B094
:1008400083B9264A1068516802AB03C308230DEB35
:1008500003022349234803F07FF9044620B92248C4
:1008600000F050FC002035E000F10802154604AE0F
:10087000183428686968334603C30835A5421E4604
:10088000F7D10699B1F5E02F03D9184800F03AFCEA
:10089000E8E702F1774202F57F0210398C1A002056
:1008A000104900F07BFC294606462246002000F055
:1008B00075FC04998E4202D1059B984206D00090A7
:1008C0003346059A0A4800F01DFCCBE7094800F0C2
:1008D00019FC012008B070BDC83500203C3C000860
:1008E000E8FF060000000108443C0008503C0008F6
:1008F000623C00088B3C00082DE9F04FAFB006AF1A
:1009000080460D4600F048FF0446002875D12B7E36
:10091000022B21D1EB8A012B1ED100F03BFC81463A
:10092000FFF7D8FD07EE900A9FEDA97AA94EF8EEE1
:10093000676A09F51670C6EE877A9FEDA77A67EEAB
:10094000877AFCEEE77A17EE903A03443360EB7E49
:1009500093B9A24B00221A70A437BD46BDE8F08FB0
:1009600007F10C031C440094002308224FEAC9013C
:10097000284600F0FFFF4C46AB8A013BA3425FFADA
:1009800084F90BD904F10109B9F1110FE8D1944BA5
:10099000944A40F22B11944803F0B0F807F11C0080
:1009A000FFF7B0FD224607F11C0107F10C0003F030
:1009B000C3F803460028CCD1B9F1100F07D0874BFC
:1009C00083F800903368A3F516733360C4E707F12A
:1009D000A002014602F8950D28460092072200F079
:1009E000C9FFF97A7F2904DD804B7E4A4FF4A1715B
:1009F000D1E7404600F0B4FEAEE7EB8A052B00F0ED
:100A00002F8106D8012BA7D129464046FFF74AFE81
:100A1000A2E7282B3DD0302B9ED16B7E744C013346
:100A2000627BDBB29342EA4640F01881EA7E237B88
:100A30009A4240F0138107F1A003002623F8846D49
:100A40001022009331460123284600F093FFB5F8A9
:100A50001480A8F102081FFA88F808F1030323F0B4
:100A600003030A3323F00703ADEB030D0DF118095F
:100A700033469BB2B11C98454FEAC10106F101060D
:100A80006DDD4B44009308220023284600F072FFDE
:100A9000EEE7AB8A013B9BB2C92B3FF65DAF544EEC
:100AA000347B4CBB06F10C030093082223462146FD
:100AB000284600F05FFFAB8A04F10109013BE4B274
:100AC0009C424FEAC90109DA0E34344400940023F1
:100AD0000822284600F04EFF4C46ECE70023002297
:100AE000C6E900230023B36086F8D730C6F8D830B3
:100AF000337B0BB9EB7E3373002407F11C0607F13F
:100B00000C03082221463046FC603C617C6101F008
:100B1000CDF83B7C04F10109A3424FEAC90107D992
:100B20007B6908222344304601F0C0F84C46F0E7C8
:100B3000C1F3CF010023E87E059104960393AB7EB9
:100B40000293193528230146009301951EA3D3E98A
:100B50000023404600F07AFEFFF7E4FCFCE694F840
:100B6000D70000F089FAD4F8D83006461BB994F8BB
:100B7000D70000F091FAD4F8D83043449E4204D212
:100B800094F8D700013000F087FA1A4B4FEA980B1F
:100B90000025AAB25A4510462EDA5AB994F8D72041
:100BA00042B9D4E900120A4304D1D9F800201A60EE
:100BB0000135EEE7226859F820107B6002EB8000D7
:100BC00000F04AFA7B68F3E726417272DF25D7B757
:100BD00000FF7F47A03500200000C8439D3500205E
:100BE0009C3C0008483D0008F53C0008173D000803
:100BF000C835002000250020D4E90023D4F8D850BF
:100C000012EB080043F10001C4E90001454494F8E7
:100C1000D700C4F8D85000F02FFA854209D394F8D1
:100C2000D730013384F8D730D4F8D8309E1BC4F8BD
:100C3000D860B8F1FF0F0ADC104B00201968207350
:100C400000F00AFAFFF7F8FD08B1FFF7F7FB236899
:100C50000B4A9B0A013313810023A360D5467BE630
:100C6000BFF34F8F0749084BCA6802F4E062134391
:100C7000CB60BFF34F8F00BFFDE700BF0025002012
:100C80009025002000ED00E00400FA0508B54FF0C3
:100C900000530B4A196891420AD10A4A597D1170D2
:100CA00009481B7D0373C92208490E3000F010FA71
:100CB000E02200214FF00050BDE8084000F01ABAD1
:100CC0009AAD44C504250020C83500201600002038
:100CD0001FB501231F498DF80B3000240622ADF803
:100CE0000C401D488DF80C304FF005134B60ADF8EB
:100CF00008208DF80A2001F0BFFD184B0093184919
:100D0000184B01944FF48052174800F0F3FC174B36
:100D1000197811B1144800F023FD00F03BFA0446A5
:100D2000FFF7D8FB07EE900A9FED117AF8EE676A9D
:100D300004F51670C6EE877A9FED0E7A67EE877A15
:100D4000FCEEE77A17EE903A034418460A4B186017
:100D500004B010BD08250020B8360020B1050008F9
:100D60009C250020F9080008A43500200425002057
:100D700000FF7F470000C843A03500202DE9F04F59
:100D80009DA7D7E900670FF27829D9E90089934C2C
:100D900093B0DFF874B2DFF874A2204600F0A2FD31
:100DA0000CAD079098B310220021284600F0A2F95C
:100DB000079B197B4FF0000261F3030219468DF87F
:100DC000302051F8040F49680EAA03C21B680D9A1F
:100DD00063F31C029DF830300D9243F020038DF830
:100DE000303000232A461946584601F055FD079039
:100DF00030B9204600F07AFD079B8AF80030CCE736
:100E00009AF80030072B40DC01338AF800301822B2
:100E10000021284600F06EF9DFF8ECB1DFF8F0A110
:100E2000002319462A46584601F05EFD014680BB64
:100E3000102208A800F05EF9DAF8143083F4805329
:100E4000CAF8143000F0A8F90B4612A9024611E9BD
:100E500003000DF1240E8EE803009DF83410C1F359
:100E6000030089064CBF0E99BDF838108DF82C0090
:100E700046BFC1F31C0141F00041C1F30A010891D2
:100E8000204608A900F078FFCAE7204600F02EFDB2
:100E9000BDE7204600F080FC8246002852D100F0D9
:100EA00079F94F4B1A6890424CD3079300F072F9CE
:100EB0008346FFF70FFB07EE900A9FED4A7A8DF805
:100EC00020A0F8EE676A0BF51670C6EE877ADFF899
:100ED00044B19BF800109FED447A67EE877AFCEEF0
:100EE000E77A17EE903A03441846079B186011B949
:100EF00001238DF8203028460791FFF703FB07995F
:100F0000C1F1100A5FFA8AFABAF1060F28BF4FF052
:100F1000060A524629440DF1210000F0D9F80AF1E1
:100F20000103049308AB0393182302932F4B0193FF
:100F30000123009332463B46204600F02FFC00235D
:100F40008BF8003000F026F9294ADFF8CCA01368AE
:100F5000C31AB3F57A7F31D3106000F01DF9024651
:100F60000B46204600F0C8FC204600F015FC28B3D4
:100F70009AF80C30DFF8A4B0002B18BF03238BF8CD
:100F8000053000F007F94FF47A732946B0FBF3F00F
:100F9000CBF800005846FFF74FFB182307300293A9
:100FA000144B0193C0F3CF0040F25513049000930B
:100FB000039542464B46204600F0F0FB9AF80C3071
:100FC0000BB1FFF7AFFA9AF80C30002B7FF4E1AECB
:100FD00013B0BDE8F08F00BFAFF30080A435002050
:100FE000A035002000FF7F470000C8439C3500204B
:100FF000A8360020AC360020401DA12026812A0BF7
:10100000F1C6A7C1D068080FB8360020AD36002061
:10101000000402409D350020C835002090250020A6
:1010200070B502F077F8094C094E20700025306841
:101030002378834208D902F067F833680544013306
:10104000B5F5803F3360F2D370BD00BFB4360020E9
:10105000B036002002F00EB907B502AB00F1006017
:1010600043F8041D0422194600F5803002F098F878
:1010700003B05DF804FB0000054B1A68054B1B78B4
:101080009B1A834202D9104402F03EB800207047F8
:10109000B0360020B436002038B5074D0446286825
:1010A000204402F039F828B928682044BDE83840C7
:1010B00002F04AB838BD00BFB0360020022802BF97
:1010C000024B4FF080529A61704700BF000402400B
:1010D00010B50023934203D0CC5CC4540133F9E72C
:1010E00010BD000002460346981A13F9011B00299F
:1010F000FAD1704702440346934202D003F8011B21
:10110000FAE770470FB4002004B070470EB4002017
:1011100003B07047FEE7000000B59BB0EFF3098114
:1011200068226846FFF7D4FFEFF30583034B9A6B01
:101130009A6A9A6A9A6A9A6A9B6AFEE700ED00E0E8
:1011400000B59BB0EFF3098168226846FFF7C0FF46
:10115000EFF30583044B9A6B9A6A9A6A9A6A9A6AC1
:101160009A6A9B6AFEE700BF00ED00E000B59BB005
:10117000EFF3098168226846FFF7AAFFEFF30583C2
:10118000034B5A6B9A6A9A6A9A6A9A6A9B6AFEE752
:1011900000ED00E002F0B8B802F0A2B810B5074CBC
:1011A0000A44914208D011F8013B4340DBB254F8A5
:1011B000233083EA1020F4E710BD00BF8C3D000807
:1011C0000246006848B103681360D388118901336F
:1011D0009BB29942D38038BF1381704770B588B0F5
:1011E0000D460446202200216846FFF783FF204673
:1011F0000495FFF7E5FF054658B16B46044608AE77
:101200001A4603CAB24220606160134604F1080422
:10121000F6D1284608B070BD2DE9F04130B9274B12
:10122000274A40F2C531274802F068FC0B7C23B9FD
:10123000254B234A40F2C631F5E7C66986B9C1613C
:10124000BDE8F081002B29DA930CAB4229D1B442DE
:1012500001D10C60F3E7C8F800100C60BDE8F08124
:101260004B6823F06047BD0C4FEAD37EC3F3807C0C
:1012700015EA230538BF3D46B04634466368BEEBE9
:10128000D37F23F06042DDD1974203D1C3F3807353
:101290009C450AD1974205E01C46EFE7AA4206D0DA
:1012A00013469D422CBF00230123002BCFD123687E
:1012B000A046002BF0D12160BDE8F0811C4400085D
:1012C00010420008D4440008F544000808B5034A59
:1012D000034B044840F25E3102F010FCEC41000880
:1012E00094440008D444000808B503680B60C38820
:1012F000016033B9044B054A05484FF4C76102F059
:10130000FDFB013BC38008BD644400086042000847
:10131000D444000870B50C4600F10C05616831B981
:10132000E38A61F30903E3820020002170BD0E68A7
:101330002846FFF7D9FF6660F0E7000008B542686D
:1013400032B10B4B0B4A0C4840F22F4102F0D6FB56
:10135000C37DC3F38401013161F38603C375C38A7E
:1013600062F30903C3821B0A62F3C713C37508BD86
:10137000B04400081C420008D44400082DE9F0479E
:10138000089E32B91F4B204A204840F2395102F0E2
:10139000B5FB01F007054FEAD6082A4406F0070618
:1013A00000EBD1004FF47F49954201D1BDE8F087B1
:1013B00005F0070E06F0070AD645774638BF5746B0
:1013C000C7F10807511BEC088F4228BF0F46045D88
:1013D00008EBD60104FA0EF413F801C029FA07FE4F
:1013E00024FA0AF45FFA8EFE8CEA04044EFA0AFE2E
:1013F00004EA0E048CEA040C03F801C03D443E44A8
:10140000D2E700BF3044000834420008D44400084A
:101410002DE9F04106460F4600254FF6FF7441F2D4
:1014200021082A4630463946FEF7DAFEC0B284EA81
:101430000024082314F4004F4FEA4404A4B203F13B
:10144000FF3318BF84EA080413F0FF03F2D1083514
:10145000402DE6D12046BDE8F081000010B50A44D9
:1014600041F22104914200D110BD11F8013B80EA04
:101470000320082310F4004F4FEA400080B203F12C
:10148000FF3318BF604013F0FF03F3D1EAE7000019
:101490002DE9F04F85B08A468DE80C00BDF83C4040
:1014A000814630B9494B4A4A40F26E31494802F010
:1014B00025FB11F0604F04D0474B454A40F26F3195
:1014C000F4E7009B002B7ED024B10E9B002B7AD03A
:1014D000072C28D809F10C00FFF772FE054628B941
:1014E0006FF00205284605B0BDE8F08F14220021F8
:1014F000FFF700FE22460E9905F10800FFF7E8FD10
:10150000631C2B74009B1B782C4403F01F0363F0B7
:101510003F0323724AF000436B6029464846FFF7B9
:101520007BFE0125DEE7019B1B0A4FF000080293BA
:1015300000F10C034FF0800B464645460393039899
:10154000FFF73EFE07460028CAD014220021FFF70D
:10155000D1FDB6BB9DF804303B729DF808307B721C
:1015600002220E9B711E1944B4420AD9B8180132E6
:10157000D2B211F801EF80F808E00136072AB6B2BE
:10158000F2D1009B197801F01F01B44208BF4FF05F
:10159000400BB81841EA48114BEA010303720132CB
:1015A0004AF000437B603A7439464846FFF734FE00
:1015B0000135B4422DB288F001084FF0000BBED1C6
:1015C00090E70022CDE76FF001058BE71C4400088F
:1015D00000420008D4440008404400082DE9F047C8
:1015E0001E46CB8A9146C3F30902062A80460F465F
:1015F00019D013460021B0B28DB25A1992B2052A01
:1016000009D9A84210D8FA8A034463F30902FA827E
:101610000120BDE8F087A842F3D93A4419F8014007
:1016200094760131E8E70025FB8A7C68C3F3090062
:10163000821F1C23B2FBF3FA03FB1A2A1FFA8AF259
:101640007CB301212368002B39D1B31F03441C2034
:10165000B3FBF0F301339BB299420CD2BAF1000F05
:1016600009D14046FFF7ACFD08B1C0F800A02060EA
:1016700008B304460022B6B24FF0000AB54230D299
:10168000691E49441346E01801339BB211F801EF7B
:1016900080F804E001351C2BADB214D0AE42F2D874
:1016A000ECE74046FFF78CFD044608B100230360D9
:1016B0007C60002CDED16FF00200BDE8F0870131C4
:1016C00089B21C46BEE7AE42D8D94046FFF778FD46
:1016D00008B1C0F800A020600028ECD00446002229
:1016E000CCE7FB8AC3F30902164466F30903FB82C5
:1016F0008EE70000F8B50E4615461F46044628B989
:10170000144B154A15484F2102F0F8F92422002104
:10171000FFF7F0FC069B6360079B23626A094FF6A4
:10172000FF739A424FF0000028BF1A46A76020704E
:10173000A061E06197B204F10C05824205D100235B
:101740002B6027826382A382F8BD2E60013035466C
:101750002036F2E7184400088C410008D444000801
:1017600008B528B9084B094A7321094802F0C6F99F
:10177000037823B94BB2002B01DD017008BD054B86
:10178000024A7D21F1E700BF1C440008984100088F
:10179000D444000860430008007870472DE9F743FF
:1017A0000D9EBDF828900B9D9DF83040BDF8388007
:1017B00007461946104616B9B8F1000F43D11F2C41
:1017C00041D83B78D3B9B8F1070F39D839F00303C2
:1017D00039D1424631464FF6FF70FFF73FFE4FEAE0
:1017E000092920F0010009F44079400449EA046421
:1017F000400C44EA40244FF6FF730DE043EA09230E
:10180000B8F1070F43EA0464F5D9FFF701FE424639
:101810003146FFF723FE03468DE840012A46214664
:101820003846FFF735FE0DB9FFF750FD2B78013331
:10183000DBB21F2B88BF00232B7003B0BDE8F08301
:101840006FF00300F9E76FF00100F6E72DE9F743C9
:101850000E9F0B9D9DF83480BDF83C6081469DF83D
:10186000300007B9C6BB1F2836D899F800E0BEF192
:10187000000F34D00C0244F080049DF8281044EA94
:10188000C83444EA014444EA0E04072E44EA0064E2
:1018900015D919461046FFF7BBFD32463946FFF70A
:1018A000DDFD0346019600972A4621464846FFF78C
:1018B000EFFDB8F1010F0CD125B9FFF707FD4FF689
:1018C000FF73EFE72B780133DBB21F2B88BF0023B8
:1018D0002B7003B0BDE8F0836FF00100F9E76FF003
:1018E0000300F6E7C06900B104307047C1690B68B6
:1018F000C3610C30FFF7F8BC2DE9F84FD0F818A001
:10190000DFF86C80054616461F4654464FF0000926
:1019100000F10C0B0CB9BDE8F88FD4E90223B21A20
:1019200067EB0303994508BF90451FD2AB699C4202
:10193000214628460DD1FFF7EDFCAB691B68AB6172
:1019400021465846FFF7D0FCAC692346A2461C4608
:10195000E0E7FFF7DFFC2368CAF80030214658466D
:10196000FFF7C2FC5446DAF80030EFE72368EDE7F2
:1019700080841E002DE9F04F8BB00D46144607936E
:10198000DDF850908246002800F06481B9F1000F24
:1019900000F06081531E3F2B00F25C81012A03D1CD
:1019A000079B002B40F05681BAF81460F600002324
:1019B000B5420893099380F053812B199E420AD2B5
:1019C000761B16F0FF0607D1AB4BAC4A40F26751CD
:1019D000AB4802F093F82646DAF80C3023B9DAF86F
:1019E0001030002B00F0A5802F2D31D8C5F1300824
:1019F00046454FF000032CBF5FFA88F8B0460093CD
:101A0000294608AB4246DAF80800FFF7B7FCA6EB18
:101A100008074544FFB2BAF8143003F10053063BFF
:101A2000DB000293DAF80C3005934FF0300B059B86
:101A3000002B51D087B9DAF81000002861D0002FB0
:101A40005FD0AB4550D98F4B8C4A40F2A651BFE7CF
:101A500037464FF00008DEE7029B23B98A4B874ADE
:101A60004FF4B161B4E7029BE02B28BFE02306935B
:101A70005B44AB4204931DD95B1B9F4226BFDBB284
:101A800003930397AB4504D97E4B7C4A40F29151B6
:101A90009EE70598CDF8008008ABA5EB0B01039AF3
:101AA0000430FFF76BFC039B9844FF1A1D445FFA58
:101AB00088F8FFB2049B9B4504D3744B6F4A40F2F5
:101AC0009B5185E7029B069ADDF810B09B1A0293A2
:101AD000059B1B680593AAE7029BBB42ABD26C4BEC
:101AE000664A40F2A15173E7CDF800803A46A5EB73
:101AF0000B0108ABFFF742FCB8443D445FFA88F89D
:101B00000027BAF81430B5EBC30F04D9614B5B4A18
:101B100040F2B1515CE7B8F1400F04D95E4B574A2F
:101B200040F2B25154E767B15C4B544A40F2B351B2
:101B30004EE70093324608AB2946DAF80800FFF773
:101B40001DFC731E3F2B35B201D8A64204DD544B59
:101B5000544A40F235213BE760070AD00AAB03EB59
:101B6000D401624211F8083C02F00702134101F867
:101B7000083C082C21D9102C21D9202C8CBF0823FB
:101B80000423079A002A6DD0B4EBC30F6CD0082C45
:101B900004F1FF3215D89DF8203023FA02F2D10764
:101BA00006D54FF0FF3202FA04F423438DF82030BB
:101BB0009DF8203089F800304EE00123E1E7022350
:101BC000DFE7102C11D8BDF8203023FA02F2D2073B
:101BD00006D54FF0FF3202FA04F42343ADF820306B
:101BE000BDF82030A9F8003036E0202C0ED8089936
:101BF00021FA02F2D30705D54FF0FF3303FA04F4BC
:101C00000C430894089BC9F8003025E0402C1CD0F8
:101C1000DDE9086730463946FEF7E2FA002100F0B8
:101C2000010050EA01030BD0224601200021FEF7FB
:101C3000E3FA404261EB410106430F43CDE90867F7
:101C4000DDE90823C9E9002306E0174B154A4FF4E4
:101C50002071BDE66FF0010528460BB0BDE8F08F9E
:101C60001D46F9E7012CA3D0082CA1D9102CB7D917
:101C7000202CE5D8C6E700BF6C42000844420008AB
:101C8000D44400088E4200087B420008B34200089A
:101C9000DB420008024300083043000848430008C4
:101CA00062430008C44100086043000830B585B0B5
:101CB00030B9244B244A40F2B121244801F01EFFE0
:101CC00023B9234B204A40F2B221F6E7402A04D937
:101CD000204B1D4A40F2B621EFE722B91D4B1A4AAC
:101CE0004FF42F71E9E70024012A0294039417D1DD
:101CF0001B788DF8083053070AD004AB03EBD203EE
:101D0000554213F8084C05F00705AC4003F8084CA1
:101D100000910346002102A8FFF730FB05B030BD5B
:101D2000082AE5D9102A03D81B88ADF80830E2E765
:101D3000202A02D81B680293DDE7D3E90045CDE9EC
:101D40000245D8E79C430008D8410008D444000865
:101D5000B74300086043000870B50C4600F10C055D
:101D6000E16819B9A1602161A18270BD0E682846A1
:101D7000FFF7BAFAE660F3E72DE9F04FD1F80090EB
:101D800091B0C9F3C01604460D46CDE90223002EDA
:101D900050D0C9F3C03BC9F30626B9F1000F80F259
:101DA0009F8119F0C04F40F09B812B7B002B00F0EE
:101DB0009781BBF1020F03D02278B24240F09381A9
:101DC00009F07F02BBF1020F059236D119F07F0FA7
:101DD000C9F30F2A01D10AF0030A2B447606059AAB
:101DE00093F8038046EA0B4646EA82465FEAD81338
:101DF00046EA0A06069300F09A800022002310A902
:101E000061E90823059B009367685B4652462046BC
:101E1000B847002800F08880A7698FB9314604F1DF
:101E20000C00FFF7DBF90746D0B96FF0020011B0E4
:101E3000BDE8F08F4FF0020BAFE7C9F3074ACCE7DC
:101E40003B699E420DD03F68002FF9D1314604F125
:101E50000C00FFF7C3F907460028E6D0A3693B60F2
:101E6000A761DDE90801FFF7D3FAB882F97D08F030
:101E70001F06C1F38401711A89B20FFA81FED7E9F6
:101E80000223BEF1000FB8BF01F1200EC9F30461B7
:101E9000B8BF0FFA8EFE079152EA030100F02F81BE
:101EA000DDE90201801A61EB030102460B469F48FF
:101EB0000021994208BF9042C0F02181069B002B6F
:101EC0003FD0BEF1010F00F31A8118F0400F38D057
:101ED000DDE90223C7E90223202200210DEB0200E5
:101EE000FFF708F9DDE90223CDE908232B1D0A934A
:101EF0002B7BADF836A0013BDBB2ADF834309DF85A
:101F00001C308DF83A309DF814308DF83B30204667
:101F10008DF838B08DF83960A36808A9984738461D
:101F2000FFF70CFA002082E76FF00B007FE7A7694C
:101F300017B96FF00C007AE73B699E4296D03F6874
:101F4000F6E7FB7DC8F34012B2EBD31F40F0CE8022
:101F5000C3F38403B34240F0CC8006992B7B4FEA55
:101F6000981279B3D2073CD4032B40F2C580DDE947
:101F70000223C7E902232B7BAE1D033BDBB23246B3
:101F8000394604F10C00FFF729FB002808DA39462E
:101F90002046FFF7BFF93846FFF7D0F9032046E7A0
:101FA000AB883B832A7B033AD2B2B88A3146FFF72B
:101FB00055FAFB7DB882DA43C2F3C01262F3C7134D
:101FC000FB75AFE76AB92E1D013BDBB232463946DD
:101FD00004F10C00FFF702FB0028D8DB2A7B013A52
:101FE000E2E7FA8AC2F30902013B052AD9B250D8C6
:101FF000281D002399420AD907EB020E013210F87E
:1020000001CB8EF81AC00133062ADBB2F2D1DDE92A
:1020100002898B4207F11A02CDE908890A9238BF7A
:1020200004337A680B9234BF5B1900230C93FB8A4C
:10203000ADF836A0C3F3090319449DF81C308DF8A0
:102040003A309DF814308DF83B300023ADF8341051
:102050008DF838B08DF839607B602A7BB88A013AF8
:10206000291DFFF7FBF93B8BB882834203D1A3689C
:1020700008A92046984708A92046FFF76DFE384674
:10208000FFF75CF9B88A3B8B984214BF11200020FF
:10209000CDE6786810B34FF0060E03689BB9A2EB4B
:1020A0000E021B2A13D80332024405F1040E1F301E
:1020B0009942ACD91EF801CB02F801CF013390420E
:1020C000DBB2F5D1A3E70EF11C0E1846E5E7184B7D
:1020D000184A194840F2B31101F010FD034696E783
:1020E0006FF00900A3E66FF00A00A0E66FF00D00A4
:1020F0009DE66FF00E009AE66FF00F0097E6FB7D0D
:1021000068F386036FF3C713FB7539462046FFF764
:1021100001F9069B002B7FF4D8AEFB7DC3F384024C
:10212000013262F38603FB7503E700BF80841E0063
:10213000CC430008B0410008D4440008026843685A
:102140001143016003B11847704700002DE9F041C9
:10215000504EB04240F089804F4CDFF840E1256C92
:1021600045F000752564256E45F000752566246EE2
:10217000446DD4F8007207EA0E0747F00107C4F86F
:102180000072D4F8005205EA0E0545F0010545EA53
:102190000121C4F80012002A69D00021C4F81C12E1
:1021A0000F46C4F80412C4F80C12C4F8141204EB5D
:1021B000C10501311C29C5F84072C5F84472F6D139
:1021C0004FF0000E4FF0010C964514D1426DD2F83D
:1021D0000032B04223F00103C2F8003257D12E4B37
:1021E0001A6C22F000721A641A6E22F000721A66DB
:1021F0001B6EBDE8F0819F781D8817F0010F18BF96
:10220000D4F804820CFA05F11CBF41EA0808C4F8AE
:10221000048217F0020F1EBFD4F80C8241EA0808AE
:10222000C4F80C827F0742BFD4F814720F43C4F87D
:10223000147204EBC5055F68C5F840729F68C5F865
:102240004472D4F81C522943C4F81C120C330EF10A
:10225000010EB9E7446D0021C4F81C12C4F8041241
:10226000C4F80C12C4F81412AAE7002AF2D1436D84
:102270000022C3F84022C3F84422C3F80422C3F862
:1022800014220122C3F80C22C3F81C229EE7BDE8E9
:10229000F08100BFB8360020003802400000FFFF88
:1022A000184B5A6D936810B513F00104936005D074
:1022B00013F00C0F14BF4FF480340124D90506D558
:1022C00013F4406F14BF44F4003444F00204DA0302
:1022D00006D513F4402F14BF44F4802444F00404C2
:1022E000202383F311880021074800F011FE2146C6
:1022F0000648FFF723FF002383F31188BDE8104051
:1023000001F08AB8B8360020C0360020DC36002044
:1023100038B5154C636DDD68AA0713D05A6922F0F1
:1023200002025A61202383F31188002104F1100076
:1023300000F0EEFD012104F11800FFF7FFFE00237D
:1023400083F31188EB060BD5636D1021D960202330
:1023500083F311880548FFF7F1FE002383F311880A
:10236000BDE8384001F058B8B8360020E836002003
:1023700038B5154C636D1D69AA0713D05A6922F050
:1023800010025A61202383F31188002104F1100008
:1023900000F0BEFD022104F11800FFF7CFFE00237C
:1023A00083F31188EB060BD5636D1021196120238F
:1023B00083F311880548FFF7C1FE002383F31188DA
:1023C000BDE8384001F028B8B8360020E8360020D3
:1023D00038B5144C636D5D685D602A0710D52046E2
:1023E000032200F8482B1A6822F002021A60202308
:1023F00083F311880021FFF7A1FE002383F31188E6
:102400006B070BD5636D9969202383F31188064808
:102410000904FFF793FE002383F31188BDE83840D9
:1024200000F0FABFB8360020E836002010B50F4C97
:10243000204600F005FA0E4B63650B21132000F0D7
:10244000E7F90B21142000F0E3F90B21152000F02F
:10245000DFF90B21162000F0DBF9002320461A4695
:102460000E21BDE81040FFF771BE00BFB836002056
:1024700000640040114B984210B5044609D1104B3E
:102480001A6C42F000721A641A6E42F000721A66F8
:102490001B6E636D01221A60636D5A68D20707D5FF
:1024A000626851681268D9611A60064A5A6110BDA3
:1024B0000121082000F060FCEEE700BFB8360020E4
:1024C000003802405B87010003291AD8DFE801F0D9
:1024D000020A0F14436D9B6813F0E05F14BF0120E4
:1024E00000207047436D9868C0F380607047436D6B
:1024F0009868C0F3C0607047436D9868C0F300707F
:10250000704700207047000010B503291FD8DFE88E
:1025100001F0021F2327416D8B68C3F30163183359
:1025200001EB0313107881061ED55468C0F3001127
:10253000490041EAC40141F0040100F00F00586075
:1025400090689860D268DA6041F00101196010BDAE
:10255000436D03F5C073E5E7436D03F5C873E1E729
:10256000436D03F5D073DDE79488C0F30011490093
:1025700041EA4451E1E7000001290CD003D30229CC
:1025800010D000207047436DDA68920701D11869B6
:1025900003E001207047436DD86810F0030018BFB6
:1025A00001207047436DF2E710B539B9436DD96822
:1025B00089071BD11B699B0704D110BD012915D0C8
:1025C000022948D1416DD1F8C031D1F8C401D1F808
:1025D000C8411461D1F8CC41546120240C610C69CC
:1025E000A40717D14C6944F0100412E0416DD1F8F2
:1025F000B031D1F8B401D1F8B8411461D1F8BC417F
:1026000054612024CC60CC68A40703D14C6944F009
:1026100002044C6111795C0864F304119C0864F3B2
:102620004511117189064BBF91681189DB085B0D5B
:102630004CBF63F31C0163F30A01137948BF916037
:1026400060F3030313714FEA10234FEA104058BFA1
:1026500011811370508010BD002304491A465A504E
:10266000C8180833802B4260F9D17047103700201A
:10267000026843681143016003B1184770470000C6
:10268000024AD36843F0C003D36070470010014092
:10269000024AD36843F0C003D3607047004400404F
:1026A0002DE9F041D0F85C64F7683368DA05054637
:1026B0009CB20DD5202383F311884FF400710430B0
:1026C000FFF7D6FF6FF480733360002383F3118824
:1026D000202383F3118805F1040814F02F0333D16C
:1026E00083F31188380615D5210613D5202383F3EB
:1026F000118805F1380000F031FA002846DA082187
:10270000281DFFF7B5FF4FF67F733B40F3600023B2
:1027100083F311887A060ED563060CD5202383F344
:102720001188EA6C2B6D9A4202D12B6C002B2FD1B1
:10273000002383F31188D5F86424D368002B31D0AB
:102740001069BDE8F0411847230713D014F0080FB3
:102750000CBF00218021E00748BF41F02001A20703
:1027600048BF41F04001630748BF41F480714046D3
:10277000FFF77EFFA406736805D595F86014284618
:10278000194000F08DFA3468A4B2A6E77060BEE785
:1027900027F040073F041021281D3F0CFFF768FF7A
:1027A000F760C5E7BDE8F08108B50348FFF778FF9B
:1027B000BDE8084000F030BE9037002008B503485F
:1027C000FFF76EFFBDE8084000F026BEF83B002092
:1027D00010B5094C094A2046002100F03FFA084B89
:1027E000C4F85C34074C084A0021204600F036FA51
:1027F000064BC4F85C3410BD9037002081260008D9
:1028000000100140F83B00209126000800440040E1
:1028100000F1604300F01F02400903F56143090124
:102820008000C9B200F1604083F8001300F56140F8
:1028300001239340C0F8803103607047FFF7F6BD75
:1028400000F108020123037082600023C26000F1DE
:102850001002836143604362026103634261C363A8
:10286000C36103628362C36243638363036443643B
:102870008364C3640365704710B52023044683F363
:102880001188022303704160FFF7F4FD03232370D6
:10289000002383F3118810BD2DE9F0411F46044643
:1028A0000D461646202383F3118800F1080823788B
:1028B000042B0ED029462046FFF706FE48B12046DD
:1028C00032462946FFF720FE002080F31188BDE83C
:1028D000F0813946404600F0FFFA0028E7D0002397
:1028E00083F31188BDE8F0812DE9F0411F460446CD
:1028F0000D461646202383F3118800F11008237833
:10290000042B0ED029462046FFF736FE48B120465C
:1029100032462946FFF748FE002080F31188BDE8C3
:10292000F0813946404600F0D7FA0028E7D000236E
:1029300083F31188BDE8F081F8B515468268066911
:10294000AA420B46816938BF8568761AB5420446AB
:1029500007D218462A46FEF7BBFBA3692B44A361A6
:102960000DE011D932461846FEF7B2FBAF1B3A46CE
:10297000E1683044FEF7ACFBE2683A44A261A36828
:102980005B1BA3602846F8BD18462A46FEF7A0FB4D
:10299000E368E4E783682DE9F04104469342154675
:1029A000266938BF85684069361AB5420F4606D297
:1029B0002A46FEF78DFB63692B4463610DE012D953
:1029C0003246A5EB0608FEF783FB4246B919E068DC
:1029D000FEF77EFBE26842446261A3685B1BA36072
:1029E0002846BDE8F0812A46FEF772FBE368E4E77B
:1029F00010B50A440024C361029B006040608460FB
:102A0000C160816141610261036210BD08B58269E4
:102A10004369934201D1826882B98268013282603F
:102A20005A1C42611970426903699A4201D3C36812
:102A30004361002100F060FA002008BD4FF0FF3034
:102A400008BD000070B5202304460E4683F31188AC
:102A5000A568A5B1A368A269013BA360531CA3614B
:102A600015782269934224BFE368A361E3690BB13F
:102A700020469847002383F31188284670BD3146CD
:102A8000204600F029FA0028E2DA85F3118870BDAB
:102A90002DE9F74F05460F4690469A46D0F81C9010
:102AA000202686F311884FF0000B144664B12246AD
:102AB00039462846FFF740FF034668B95146284685
:102AC00000F00AFA0028F1D0002383F31188A8EB64
:102AD000040003B0BDE8F08FB9F1000F03D00190FE
:102AE0002846C847019B8BF31188E41A1F4486F3DC
:102AF0001188DBE7C16081614161C3611144009BC2
:102B0000006040608260016103627047F8B504466E
:102B10000E461746202383F31188A568A5B1A36844
:102B2000013BA36063695A1C62611E70236962697C
:102B30009A4224BFE3686361E3690BB1204698477A
:102B4000002080F31188F8BD3946204600F0C4F912
:102B50000028E2DA85F31188F8BD00008369426934
:102B60009A4210B501D182687AB9826801328260D6
:102B70005A1C82611C7803699A4201D3C36883613D
:102B8000002100F0B9F9204610BD4FF0FF3010BD14
:102B90002DE9F74F05460F4690469A46D0F81C900F
:102BA000202686F311884FF0000B144664B12246AC
:102BB00039462846FFF7EEFE034668B951462846D7
:102BC00000F08AF90028F1D0002383F31188A8EBE4
:102BD000040003B0BDE8F08FB9F1000F03D00190FD
:102BE0002846C847019B8BF31188E41A1F4486F3DB
:102BF0001188DBE7026843681143016003B118479D
:102C0000704700001430FFF743BF00004FF0FF3360
:102C10001430FFF73DBF00003830FFF7B9BF0000A8
:102C20004FF0FF333830FFF7B3BF00001430FFF729
:102C300009BF00004FF0FF311430FFF703BF000061
:102C40003830FFF763BF00004FF0FF323830FFF736
:102C50005DBF000000207047FFF7BABD37B50F4BCE
:102C60000360002343608360C36001230446037450
:102C7000154600900B464FF4007200F15C011430D1
:102C8000FFF7B6FE00942B464FF4007204F517715F
:102C900004F13800FFF72EFF03B030BD10450008E7
:102CA00038B5C36904460D461BB904210844FFF733
:102CB000A1FF294604F11400FFF7A8FE002806DA58
:102CC000201D4FF48061BDE83840FFF793BF38BD49
:102CD000024B00221B605B609A60704760400020DE
:102CE000002303748268054B1B6899689142FBD2EC
:102CF0005A6803604260106058607047604000206E
:102D000008B5202383F31188037C032B05D0042B03
:102D10000DD02BB983F3118808BD436900221A60D6
:102D20004FF0FF334361FFF7DBFF0023F2E790E84A
:102D30000C001A6002685360F2E70000002303747D
:102D40008268054B1B6899689142FBD85A680360FA
:102D5000426010605860704760400020054B196960
:102D60000874186802681A605360186101230374BC
:102D7000FDF7E2BA6040002030B54B1C87B0054635
:102D80000A4C10D023690A4A01A800F0DDF8284651
:102D9000FFF7E4FF049B13B101A800F011F92369C8
:102DA000586907B030BDFFF7D9FFF8E76040002051
:102DB000012D000838B50C4D41612B6981689A6876
:102DC0009142044603D8BDE83840FFF789BF184652
:102DD000FFF786FF01232C61014623742046BDE8DE
:102DE0003840FDF7A9BA00BF60400020044B1A68C4
:102DF0001B6990689B68984294BF0020012070472F
:102E00006040002010B5084C236820691A682260D1
:102E10005460012223611A74FFF790FF0146206974
:102E2000BDE81040FDF788BA6040002008B5FFF704
:102E3000DDFF18B1BDE80840FFF7E4BF08BD0000A2
:102E40008260022202740022427470478368A3F1F8
:102E50007C0243F80C2C026943F83C2C426943F88D
:102E6000382C074A43F81C2CC26843F8102C022265
:102E700003F8082C002203F8072CA3F11800704770
:102E80005103000810B5202383F31188FFF7DEFFFC
:102E900000210446FFF78EFF002383F311882046AC
:102EA00010BD0000024B1B6958610F20FFF756BF91
:102EB00060400020202383F31188FFF7F3BF000058
:102EC00008B50146202383F311880820FFF754FF3B
:102ED000002383F3118808BD49B1064B42681B6982
:102EE00018605A60136043600420FFF745BF4FF03D
:102EF000FF307047604000200368984206D01A688F
:102F00000260506059611846FFF7EABE7047000042
:102F100038B504460D462068844200D138BD0368A8
:102F200023605C604561FFF7DBFEF4E7054B03F1CE
:102F300014025A619A614FF0FF32DA6100221A627C
:102F4000704700BF60400020F8B503614FF0804338
:102F5000C2605C6A194B1A46022952F8145F38BFE6
:102F60000221954206461F460AD1586198611C62AB
:102F70000560456081600819BDE8F84000F09ABA24
:102F8000186AAB68241A0C1902D3E41A2D6804E0FD
:102F90009C4202D2204400F09BFAAB689C42F4D8D9
:102FA0006B68736035601E606E60B460A9684FF036
:102FB000FF33091BA960FB61F8BD00BF6040002022
:102FC00010B41B4C234653F8141F814210D04168A3
:102FD00002680A60026851609A424FF00001C160C5
:102FE00003D0936881680B4493605DF8044B70478D
:102FF0000A68626100209A425360C86003D15DF89C
:10300000044B00F05FBA93688868034493604FF004
:103010008042206A526A121A9342E6D9991A01290B
:1030200098BF931C18445DF8044B00F051BA00BFE0
:103030006040002000207047FEE70000704700005D
:103040004FF0FF3070470000BFF34F8F024AD36844
:10305000DB03FCD4704700BF003C024008B5094BBD
:103060001B7873B9FFF7F0FF074B1A69002ABFBF3F
:10307000064A5A6002F188325A601A6822F4806265
:103080001A6008BDA0400020003C024023016745B3
:1030900008B50B4B1B7893B9FFF7D6FF094B1A699C
:1030A00042F000421A611A6842F480521A601A68AB
:1030B00022F480521A601A6842F480621A6008BDD5
:1030C000A0400020003C0240072870B513D80B4AEE
:1030D0000B4C137863B90B4E4FF0006144F823108A
:1030E00056F823500133082B2944F7D101231370DC
:1030F00054F8200070BD002070BD00BFC440002007
:10310000A440002038450008014B53F820007047C8
:103110003845000808207047072810B5044601D933
:10312000002010BDFFF7D0FF064B53F824301844A1
:10313000C21A0BB9012010BD12680132F0D1043B54
:10314000F6E700BF38450008072810B5044621D827
:10315000FFF77AFFFFF782FF0F4AF323D360C30024
:10316000DBB243F4007343F002031361136943F4C9
:1031700080331361FFF768FFFFF7A6FF074B53F893
:10318000241000F025F9FFF783FF2046BDE810402A
:10319000FFF7C2BF002010BD003C024038450008C8
:1031A0002DE9F84312F00103154640D184182E4A48
:1031B00094423CD82D4B1B6813F0010337D02C4CA4
:1031C000FFF74CFFF323E360FFF73EFF40F20127D8
:1031D000032D01D9830713D0254C0F46401A40F226
:1031E0000118EB1B0B44012B00EB0706236924D8C5
:1031F00023F001032361FFF74BFF0120BDE8F883B3
:10320000236923F44073236123693B43236151F80D
:10321000046B0660BFF34F8FFFF716FF03689E42F3
:1032200008D0236923F001032361FFF731FF002059
:10323000BDE8F883043D0430CAE723F440732361FA
:10324000236943EA08032361B94637F8023B338018
:10325000BFF34F8FFFF7F8FE3688B9F80030B6B2EB
:10326000B342BED0DDE700BFFFFF070800380240D1
:10327000003C0240084908B50B7828B153B9FFF764
:10328000EDFE01230B7008BD23B1BDE808400870B6
:10329000FFF7FEBE08BD00BFA04000204FF08043F6
:1032A00030B5586A0B4B1A6882421A460FD90A4B3E
:1032B0000A49D3E9004514F1FF3445F10005C3E99B
:1032C00000450B6803F5830303F637130B601060AA
:1032D00030BD00BFC8400020D0400020CC400020BE
:1032E00070B500F07DF90646FFF7D8FF054BD3E92E
:1032F0000045241845F10005304600F07BF92046D2
:10330000294670BDD040002038B500F069F9054667
:10331000FFF7C4FF054B4FF47A74B0FBF4F4186860
:103320000444284600F066F9204638BDCC40002011
:1033300010B50244064B0439D2B2904200D110BD00
:10334000441C00B253F8200041F8040FE0B2F4E747
:1033500050280040104B30B51C6F240407D41C6F5C
:1033600044F400741C671C6F44F400441C670B4C4D
:10337000236843F4807323600244094B0439D2B2BA
:10338000904200D130BD441C00B251F8045F43F8B4
:103390002050E0B2F4E700BF003802400070004067
:1033A0005028004007B5012201A90020FFF7C0FF07
:1033B000019803B05DF804FB07B502A9012241F8AA
:1033C000040D0020FFF7C6FF03B05DF804FB00000A
:1033D00070470000034B1B689B0042BF024B012259
:1033E0001A70704774380240D8400020014B18789A
:1033F000704700BFD8400020064A536823F00103FD
:103400005360EFF30983683383F30988002383F360
:103410001188704730EF00E010B5202383F3118846
:10342000104B5B6813F4006318D0F1EE103AEFF321
:1034300009844FF0807344F84C3C0B4BDB6844F834
:10344000083CA4F1680383F30988FFF7CFFC18B1A7
:10345000064B44F8503C10BD054BFAE783F3118846
:1034600010BD00BF00ED00E030EF00E06103000898
:103470006403000870470000FEE70000084A094B9B
:1034800009498B4204D3094A0021934205D370476E
:1034900052F8040F43F8040BF3E743F8041BF4E776
:1034A00018470008DC420020DC420020DC420020FB
:1034B00000F034B94FF08043002258631A610222B1
:1034C000DA6070474FF080430022DA6070470000F6
:1034D0004FF0804358637047FEE7000010B5174C6B
:1034E000FFF7F6FBFFF722FD802215492046FFF784
:1034F000A7FC012344F8180C0374124B124AD96834
:1035000021F4E0610904090C0A431049DA60CA6831
:1035100042F08072CA600E490A6842F001020A60F5
:103520001022DA77202283F82220002383F31188E7
:1035300062B60848BDE81040FFF7A4BC88400020F0
:103540005845000800ED00E00003FA05F0ED00E04A
:10355000001000E0604500082DE9F84F1F4C4FF0C7
:103560000008656904F11407C1464FF08043266ADC
:103570005B6AAA689E1B96421DD34FF0200AAA6878
:10358000236AD5F80CB0134423622B68BB425F60FA
:10359000A6EB02066361C5F80C8001D1FFF792FF2C
:1035A00089F311882869D8478AF311886569AB685F
:1035B0009E42E4D2D9E76269BA420CD09168236294
:1035C0008E1B9660A86802282CBF1818981CBDE8AE
:1035D000F84FFFF77DBFBDE8F88F00BF60400020C7
:1035E000EFF3118020B9EFF30583202282F31188D5
:1035F0007047000010B558B9EFF30584C4F3080410
:1036000014B180F3118810BDFFF710FC84F311880A
:1036100010BD00004B6843608B688360CB68C3605B
:103620000B6943614B6903628B6943620B680360FA
:103630007047000008B51F4B1F481A6942F0FF028F
:103640001A611A6922F0FF021A611A691A6B42F0B4
:10365000FF021A631A6D42F0FF021A65174A1B6DCA
:103660001146FFF7D7FF164802F11C01FFF7D2FF02
:10367000144802F13801FFF7CDFF134802F154015D
:10368000FFF7C8FF114802F17001FFF7C3FF1048B0
:1036900002F18C01FFF7BEFF0E4802F1A801FFF70F
:1036A000B9FF0D4802F1C401FFF7B4FFBDE80840BF
:1036B00000F09CB80038024000000240804500083D
:1036C0000004024000080240000C024000100240CA
:1036D0000014024000180240001C024008B500F02F
:1036E000FDF9FFF7FBFEBDE80840FFF773BE0000E1
:1036F000704700004FF0804310B51A69920708D553
:1037000000241C61202383F31188FFF725FF84F335
:103710001188BDE81040FFF77FBE0000104B1A6C07
:1037200042F001021A641A6E42F001021A660D4A52
:103730001B6E936843F0010393604FF080435F2258
:103740009A624FF0FF32DA6200229A615A63DA60BD
:103750005A6001225A6108211A601C20FFF758B8EC
:1037600000380240002004E01E4B1A6962F0FF029C
:103770001A611A69D2B21A614FF0FF301A695A6998
:10378000586100215A6959615A691A6A62F0805277
:103790001A621A6A02F080521A621A6A5A6A5862E7
:1037A0005A6A59625A6A1A6C42F080521A641A6E46
:1037B00042F080521A661A6E0B4A106840F480700C
:1037C0001060186F00F44070B0F5007F1EBF4FF41A
:1037D000803018671967536823F40073536000F052
:1037E0005DB900BF0038024000700040334B344ADE
:1037F0001A64344A4FF4404111601A6842F00102E1
:103800001A601A689207FCD59A6822F003029A603F
:103810002A4B19469A6812F00C02FBD1186800F086
:10382000F90018609A601A6842F480321A600B68D6
:103830009B03FCD54B6F43F001034B671F4B5A6F43
:103840009007FCD5204A5A601A6842F080721A60CC
:103850001C4A53685904FCD5184B1A689201FCD5D0
:103860001A4A9A600322C3F88C200022C3F89420DD
:10387000174B1A68174B9A42174B1BD1174A1168FE
:10388000174A914216D140F203121A600B4B9A6804
:1038900042F002029A609A6802F00C02082AFAD1F9
:1038A0005A6C42F480425A645A6E42F480425A661C
:1038B0005B6E704740F20372E7E700BF00380240DA
:1038C000000400100070004010604108009088382B
:1038D000002004E011640020003C024000ED00E004
:1038E00041C20F41084A08B5536911680B4003F003
:1038F0000103536123B1054A13680BB1506898471F
:10390000BDE80840FFF788BD003C014010370020AB
:10391000084A08B5536911680B4003F0020353616C
:1039200023B1054A93680BB1D0689847BDE80840B9
:10393000FFF772BD003C014010370020084A08B56F
:10394000536911680B4003F00403536123B1054A26
:1039500013690BB150699847BDE80840FFF75CBD9B
:10396000003C014010370020084A08B5536911682F
:103970000B4003F00803536123B1054A93690BB16F
:10398000D0699847BDE80840FFF746BD003C0140BC
:1039900010370020084A08B5536911680B4003F03E
:1039A0001003536123B1054A136A0BB1506A98475B
:1039B000BDE80840FFF730BD003C01401037002053
:1039C000174B10B55C691A68144004F478725A6198
:1039D000A30604D5134A936A0BB1D06A98476006D0
:1039E00004D5104A136B0BB1506B9847210604D5D0
:1039F0000C4A936B0BB1D06B9847E20504D5094A8A
:103A0000136C0BB1506C9847A30504D5054A936C11
:103A10000BB1D06C9847BDE81040FFF7FDBC00BF6C
:103A2000003C0140103700201A4B10B55C691A6841
:103A3000144004F47C425A61620504D5164A136DA1
:103A40000BB1506D9847230504D5134A936D0BB104
:103A5000D06D9847E00404D50F4A136E0BB1506E39
:103A60009847A10404D50C4A936E0BB1D06E9847C9
:103A7000620404D5084A136F0BB1506F98472304B2
:103A800004D5054A936F0BB1D06F9847BDE810403D
:103A9000FFF7C2BC003C014010370020062108B5EA
:103AA0000846FEF7B5FE06210720FEF7B1FE062107
:103AB0000820FEF7ADFE06210920FEF7A9FE06212B
:103AC0000A20FEF7A5FE06211720FEF7A1FE06211B
:103AD0002820BDE80840FEF79BBE000008B5FFF7B0
:103AE00043FEFEF7B9FDFEF7A9FEFFF7B5F8FFF7B5
:103AF000FFFDBDE80840FFF7DBBC00001FB51C461A
:103B0000094B1B680546D86852B1084B02928DE8F4
:103B10000A0022462B460649FDF7F8FA00F042F863
:103B2000044B1A46F2E700BF182500206046000843
:103B30006D460008993C000810B5013902449042D6
:103B400001D1002010BD10F8013B11F8014FA34234
:103B5000F5D0181B10BD00002DE9F8430746884634
:103B600091461E468BB10D46A8EB0500B54207EB0A
:103B7000000402D20020BDE8F883324649462046C0
:103B8000FFF7DAFF18B1013DEEE7BDE8F883204604
:103B9000BDE8F883034611F8012B03F8012B002A36
:103BA000F9D1704708B5062000F02CF80120FFF786
:103BB00043FA00001F2938B504460D4604D91623E0
:103BC00003604FF0FF3038BD426C12B152F8213023
:103BD0004BB9204600F030F82A4601462046BDE8A1
:103BE000384000F017B8012B0AD0591C03D1162316
:103BF0000360012038BD002442F82540284698473C
:103C0000002038BD024B01461868FFF7D3BF00BF44
:103C10001825002038B5074C0023054608461146F4
:103C20002360FFF70DFA431C02D1236803B12B6018
:103C300038BD00BFD8420020FFF7FCB940A2E4F134
:103C4000646891064E6F20617070207369670A0086
:103C5000426164206677206C656E67746820257504
:103C60000A00426164206170702043524320307822
:103C7000253038783A30782530387820307825303B
:103C800038783A3078253038780A00476F6F6420EA
:103C90006669726D776172650A000000726563651E
:103CA000697665645F756E697175655F69645F6C7F
:103CB000656E203C2055415643414E5F50524F5453
:103CC0004F434F4C5F44594E414D49435F4E4F4423
:103CD000455F49445F414C4C4F434154494F4E5F0F
:103CE000554E495155455F49445F4D41585F4C45DC
:103CF0004E475448002E2E2F2E2E2F546F6F6C736C
:103D00002F41505F426F6F746C6F616465722F63F7
:103D1000616E2E63707000616C6C6F6361746564BA
:103D20005F6E6F64655F6964203C3D20313237000F
:103D30006F72672E6172647570696C6F742E637533
:103D400061765F6770730000766F69642068616EEA
:103D5000646C655F616C6C6F636174696F6E5F72D8
:103D60006573706F6E73652843616E617264496E2E
:103D70007374616E63652A2C2043616E61726452B4
:103D8000785472616E736665722A29000000000023
:103D9000963007772C610EEEBA51099919C46D0758
:103DA0008FF46A7035A563E9A395649E3288DB0EB3
:103DB000A4B8DC791EE9D5E088D9D2972B4CB60996
:103DC000BD7CB17E072DB8E7911DBF906410B71D73
:103DD000F220B06A4871B9F3DE41BE847DD4DA1AAC
:103DE000EBE4DD6D51B5D4F4C785D38356986C13DD
:103DF000C0A86B647AF962FDECC9658A4F5C011456
:103E0000D96C0663633D0FFAF50D088DC8206E3B33
:103E10005E10694CE44160D5727167A2D1E4033C45
:103E200047D4044BFD850DD26BB50AA5FAA8B5356C
:103E30006C98B242D6C9BBDB40F9BCACE36CD8325B
:103E4000755CDF45CF0DD6DC593DD1ABAC30D92602
:103E50003A00DE518051D7C81661D0BFB5F4B42105
:103E600023C4B3569995BACF0FA5BDB89EB8022802
:103E70000888055FB2D90CC624E90BB1877C6F2F87
:103E8000114C6858AB1D61C13D2D66B69041DC7682
:103E90000671DB01BC20D2982A10D5EF8985B1715B
:103EA0001FB5B606A5E4BF9F33D4B8E8A2C907780A
:103EB00034F9000F8EA8099618980EE1BB0D6A7FA1
:103EC0002D3D6D08976C6491015C63E6F4516B6B5A
:103ED00062616C1CD83065854E0062F2ED95066C0F
:103EE0007BA5011BC1F4088257C40FF5C6D9B06584
:103EF00050E9B712EAB8BE8B7C88B9FCDF1DDD62E1
:103F0000492DDA15F37CD38C654CD4FB5861B24D46
:103F1000CE51B53A7400BCA3E230BBD441A5DF4A10
:103F2000D795D83D6DC4D1A4FBF4D6D36AE96943D3
:103F3000FCD96E34468867ADD0B860DA732D04447E
:103F4000E51D03335F4C0AAAC97C0DDD3C710550A9
:103F5000AA41022710100BBE86200CC925B5685750
:103F6000B3856F2009D466B99FE461CE0EF9DE5E99
:103F700098C9D9292298D0B0B4A8D7C7173DB3594A
:103F8000810DB42E3B5CBDB7AD6CBAC02083B8EDDB
:103F9000B6B3BF9A0CE2B6039AD2B1743947D5EAE8
:103FA000AF77D29D1526DB048316DC73120B63E317
:103FB000843B64943E6A6D0DA85A6A7A0BCF0EE476
:103FC0009DFF099327AE000AB19E077D44930FF031
:103FD000D2A3088768F2011EFEC206695D5762F728
:103FE000CB67658071366C19E7066B6E761BD4FE65
:103FF000E02BD3895A7ADA10CC4ADD676FDFB9F942
:10400000F9EFBE8E43BEB717D58EB060E8A3D6D603
:104010007E93D1A1C4C2D83852F2DF4FF167BBD131
:104020006757BCA6DD06B53F4B36B248DA2B0DD834
:104030004C1B0AAFF64A0336607A0441C3EF60DFD7
:1040400055DF67A8EF8E6E3179BE69468CB361CBC0
:104050001A8366BCA0D26F2536E2685295770CCCE5
:1040600003470BBBB91602222F260555BE3BBAC526
:10407000280BBDB2925AB42B046AB35CA7FFD7C217
:1040800031CFD0B58B9ED92C1DAEDE5BB0C2649B08
:1040900026F263EC9CA36A750A936D02A906099C3B
:1040A0003F360EEB8567077213570005824ABF95AE
:1040B000147AB8E2AE2BB17B381BB60C9B8ED29231
:1040C0000DBED5E5B7EFDC7C21DFDB0BD4D2D38688
:1040D00042E2D4F1F8B3DD686E83DA1FCD16BE81FB
:1040E0005B26B9F6E177B06F7747B718E65A0888CC
:1040F000706A0FFFCA3B06665C0B0111FF9E658F5D
:1041000069AE62F8D3FF6B6145CF6C1678E20AA006
:10411000EED20DD75483044EC2B30339612667A78C
:10412000F71660D04D476949DB776E3E4A6AD1AEDB
:10413000DC5AD6D9660BDF40F03BD83753AEBCA96A
:10414000C59EBBDE7FCFB247E9FFB5301CF2BDBDD7
:104150008AC2BACA3093B353A6A3B4240536D0BAE0
:104160009306D7CD2957DE54BF67D9232E7A66B37D
:10417000B84A61C4021B685D942B6F2A37BE0BB42A
:10418000A18E0CC31BDF055A8DEF022D63616E619A
:104190007264496E6974000063616E617264536594
:1041A000744C6F63616C4E6F64654944000000009D
:1041B00063616E61726448616E646C6552784672C8
:1041C000616D650063616E6172644465636F64650F
:1041D0005363616C6172000063616E617264456E6D
:1041E000636F64655363616C61720000696E637232
:1041F000656D656E745472616E73666572494400D4
:10420000656E717565756554784672616D6573008C
:104210007075736854785175657565007072657056
:10422000617265466F724E6578745472616E736622
:1042300065720000636F70794269744172726179CE
:104240000000000064657363617474657254726188
:104250006E736665725061796C6F61640000000076
:1042600066726565426C6F636B0000006269745F23
:104270006C656E677468203E20300072656D616900
:104280006E696E675F62697473203E203000696EEC
:104290007075745F6269745F6F6666736574203EE3
:1042A0003D20626C6F636B5F6269745F6F666673FB
:1042B000657400626C6F636B5F656E645F626974E6
:1042C0005F6F6666736574203E20626C6F636B5F20
:1042D0006269745F6F66667365740072656D6169AB
:1042E0006E696E675F6269745F6C656E6774682083
:1042F0003C3D2072656D61696E696E675F626974CD
:104300007300696E7075745F6269745F6F6666735F
:104310006574203C3D207472616E736665722D3E3B
:104320007061796C6F61645F6C656E202A20380063
:104330006F75747075745F6269745F6F66667365BC
:1043400074203C3D2036340072656D61696E696E83
:10435000675F6269745F6C656E677468203D3D20BD
:10436000300028726573756C74203E203029202639
:10437000262028726573756C74203C3D20363429E4
:104380002026262028726573756C74203C3D2062BF
:1043900069745F6C656E6774682900006465737486
:1043A000696E6174696F6E20213D202828766F69DF
:1043B00064202A2930290076616C756520213D2012
:1043C0002828766F6964202A293029006F66667371
:1043D00065745F77697468696E5F626C6F636B2088
:1043E0003C2028333255202D205F5F6275696C7444
:1043F000696E5F6F66667365746F66202843616ED1
:10440000617264427566666572426C6F636B2C20E4
:1044100064617461292900006F75745F696E73208F
:10442000213D202828766F6964202A293029000040
:104430007372635F6C656E203E2030550000000093
:104440002863616E5F6964202620307831464646D5
:10445000464646465529203D3D2063616E5F6964AE
:1044600000000000616C6C6F6361746F722D3E73AD
:104470007461746973746963732E63757272656EA7
:10448000745F75736167655F626C6F636B73203E09
:10449000203000007472616E736665725F6964201B
:1044A000213D202828766F6964202A2930290000C0
:1044B00073746174652D3E6275666665725F626CC9
:1044C0006F636B73203D3D202828766F6964202A36
:1044D000293029002E2E2F2E2E2F6D6F64756C65BE
:1044E000732F6C696263616E6172642F63616E61C8
:1044F00072642E63006974656D2D3E6672616D6530
:104500002E646174615F6C656E203E203000000097
:1045100000000000212C00080D2C0008492C000888
:10452000352C0008412C00082D2C0008192C0008FF
:10453000052C0008552C0008004000000040000039
:1045400000400000004000000000010000000200E8
:1045500000000200000002006D61696E00000000B2
:1045600078450008E0400020D8420020010000000B
:10457000D93400080000000069646C650000000088
:10458000A000002800000000AAAAAAAA500000006B
:10459000FFFF0000007700000000000000A40A01F7
:1045A00000000000AAA6AAAA80500000DFEF0000C9
:1045B00000000077880000000000000000000000FC
:1045C000AAAAAAAA00000000FFFF00000000000045
:1045D000000000000000000000000000AAAAAAAA33
:1045E00000000000FFFF00000000000000000000CD
:1045F0000000000000000000AAAAAAAA0000000013
:10460000FFFF0000000000000000000000000000AC
:1046100000000000AAAAAAAA00000000FFFF0000F4
:10462000000000000000000000000000000000008A
:10463000AAAAAAAA00000000FFFF000000000000D4
:104640000000000000000000000000000A00000060
:104650000000000003000000000000000000000057
:104660002C2066756E6374696F6E3A2000617373F7
:10467000657274696F6E2022257322206661696CF1
:1046800065643A2066696C6520222573222C206CB3
:10469000696E65202564257325730A0000000000FB
:1046A000FFFFFFFF74000000640000000000000036
:1046B000FE2A0100D20400001C250020000000009A
:1046C00000000000000000000000000000000000EA
:1046D00000000000000000000000000000000000DA
:1046E00000000000000000000000000000000000CA
:1046F00000000000000000000000000000000000BA
:1047000000000000000000000000000000000000A9
:0C4710000000000000000000000000009D
:00000001FF
